:10000000ED2880308D00FE30A7200130A72075300C
:1000100092003030B8288D018D179A009A08031D80
:1000200013280301142801309A0203108E0C8E0C41
:100030008E0CC0300E05403E9A07FE30A7201A08ED
:10004000A7288D018D179A00FE30A7201A08A7282F
:100050009001950096018C11100803198C1505303C
:100060008F00273094001030412003309400E83096
:10007000412094016430412094010A304120150848
:10008000482893001608920015089100CC2011080A
:1000900091008F0303198C111008031952280F02C5
:1000A000031859281108031D8C118C195928303E4A
:1000B000A7280800980005108510831605108510E4
:1000C0000F308605831218088C1884283E30920061
:1000D0008030B82033309700982013309200883059
:1000E000B82098206430B72098206430B7202230A0
:1000F00097009820283083200C30832006308320FE
:100100008C14180884280C1497000C1C9228851055
:10011000033C031C9728972007309200D030B8206A
:10012000031408000C14FE3C0319A52885140C1CAC
:100130000C1005140F3086051708F03986040510D9
:10014000970E0C1898283230B7201808E8288D1B15
:100150005A28080094019300FF309307031C94076A
:10016000031CE82803309200DF30B820AC2892014D
:10017000E83E91009209FC30031CC1289107031846
:10018000BE2891070000920FBE281118C728911CA5
:10019000CB280000CB28080096019501103097006D
:1001A000120D950D960D130895021408031C140FDB
:1001B00096020318E2281308950714080318140F71
:1001C00096070310910D920D970BD0281108E8287F
:1001D000831383120313000008008C018316061496
:1001E0008614061586150516013083129400F43026
:1001F000AB20FE305A2001305A2080308D008030F4
:10020000212054305A2042305A2032305A204E3069
:100210005A2048305A2044305A2003309400E830A5
:10022000AB2080308D00C030212044305A20543023
:100230005A204D305A2046305A2020305A2044301F
:100240005A2045305A2043305A204F305A204430EB
:100250005A2045305A2052305A2003309400E8305A
:10026000AB20012001309E009D019F01051E392910
:100270003A293629861D3D299F0A061D412902304B
:100280009F07861C452904309F07061C4929083012
:100290009F0710301D02031D4F299E0A9D010F303C
:1002A0001D020130031D00309C0002301E0201308F
:1002B000031D00301C0503195E2931299D0A0A30EF
:1002C0001F02031D6D2980308D001E088E001D0841
:1002D0000D2030305A209F01CB290B301F02031D07
:1002E0007B2980308D001E088E001D080D202A30CD
:1002F0005A209F01CB290C301F02031D8929803011
:100300008D001E088E001D080D2023305A209F01ED
:10031000CB290D301F02031D972980308D001E0848
:100320008E001D080D2041305A209F01CB290E3030
:100330001F02031DA52980308D001E088E001D0898
:100340000D2042305A209F01CB290F301F02031D80
:10035000B32980308D001E088E001D080D2043300B
:100360005A209F01CB299F08031DC02980308D0092
:100370001E088E001D080D2044305A209F01CB29F5
:1003800080308D001E088E001D080D200130900069
:100390001F0829209F01051ECE29CB29362963007D
:0203A000CF2963
:02400E00F13F80
:00000001FF
